:100000000C9439000C9456000C9456000C94560035
:100010000C9456000C9456000C9456000C94560008
:100020000C9456000C9456000C9456000C945600F8
:100030000C9456000C9456000C9456000C945600E8
:100040000C9456000C9456000C9456000C945600D8
:100050000C94560005A84CCDB2D44EB93836A9023E
:100060000C50B9918688083CA6AAAA2ABE000000B6
:10007000803F11241FBECFE5D4E0DEBFCDBF10E02E
:10008000A0E6B0E0E8EBFCE102C005900D92A03ED6
:10009000B107D9F712E0A0EEB0E001C01D92A4387C
:1000A000B107E1F70E944B030C945A0E0C94000028
:1000B000CF93DF9300D0CDB7DEB7AD98811102C0EA
:1000C000AC9801C0AC9AAD9A25B3862F992787FDCD
:1000D0009095807F99279595879595958795959586
:1000E000879595958795922F907F892B85BBAD98A5
:1000F000AD9A85B36F70807F682B65BBAD9821E2A8
:10010000249FC001259F900D11249A8389838981A2
:100110009A81892B49F089819A8101979A838983F1
:1001200089819A81892BB9F70F900F90DF91CF9138
:100130000895CF93DF93FC016081662351F0EC01B9
:10014000219642E050E081E00E94580069916111DF
:10015000F8CFDF91CF91089544E050E068E280E06D
:100160000E94580044E050E068E280E00E9458009D
:1001700044E050E068E280E00E94580048EC50E023
:1001800062E080E00E94580044E050E06CE080E0D3
:100190000E94580040E850E061E080E00E94580072
:1001A00044E050E066E080E00E94580008958A3004
:1001B00040F4682F605D42E050E081E00E9458000A
:1001C0000895682F695C42E050E081E00E94580089
:1001D0000895CF93C82F82958F700E94D7008C2FDF
:1001E0008F700E94D700CF910895CF93C82F892F89
:1001F0000E94E9008C2F0E94E900CF910895CF93CF
:10020000DF93C82FD9E28D9FD12D1124D295DF70B5
:100210006D2F605D42E050E081E00E94580084E66E
:10022000D89FC0191124DDECCD9FD12D1124D69576
:10023000D695D6956D2F605D42E050E081E00E943A
:100240005800DD0F8D2F880F880FD80FCD1B6C2F16
:10025000605D42E050E081E00E945800DF91CF9164
:1002600008950F931F93CF93DF938C019C013295D8
:1002700022952F7023273F702327A7E4B3E00E9425
:100280002B0EEC01D695C795D695C795D695C795F3
:100290006C2F605D42E050E081E00E94580020E158
:1002A00037E2C29FC001C39F900DD29F900D1124D1
:1002B000081B190B98013695279536952795369585
:1002C0002795A5ECB0E20E942B0EEC01D295C295C9
:1002D000CF70CD27DF70CD276C2F605D42E050E0FE
:1002E00081E00E94580028EE33E0C29FC001C39F06
:1002F000900DD29F900D1124081B190B9801369573
:10030000279536952795ABE7B4E10E942B0EEC01BB
:10031000D695C7956C2F605D42E050E081E00E9469
:10032000580024E62C9FC0012D9F900D1124081B1E
:10033000190B9801ADECBCEC0E942B0EEC01D6958C
:10034000C795D695C795D695C7956C2F605D42E049
:1003500050E081E00E945800CE01880F991FCC0F19
:10036000DD1FCC0FDD1FCC0FDD1FC80FD91F0C1BED
:100370001D0B602F605D42E050E081E00E9458005C
:10038000DF91CF911F910F910895EF92FF920F93FC
:100390001F93CF93DF9300E0C0E0D0E0F12C16C0B4
:1003A000612F6E2944E050E08F2D0E9458004AE0F2
:1003B00050E0602F81E00E9458001F5F183081F7E5
:1003C000069500612196C530D10569F09E01220F86
:1003D000331F220F331F220F331F6894EE24E6F8D9
:1003E000E22A1F2DDDCFDF91CF911F910F91FF905A
:1003F000EF9008959F92AF92BF92CF92DF92EF92CB
:10040000FF920F931F93CF93DF93E12CF12CA12C3C
:10041000B12C0F2EF7E0CF2ED12CF02D22C06C2F57
:10042000692944E050E080E00E9458000C171D0745
:100430003CF04AE050E060E081E00E94580006C0D5
:100440004AE050E06FEF81E00E9458002196C830EA
:10045000D10529F78FEFE81AF80A88E0E816F104C9
:1004600081F0C701880F991F880F991F880F991F66
:100470006894992496F8982AE50186010E191F09B7
:10048000CECFDF91CF911F910F91FF90EF90DF9032
:10049000CF90BF90AF909F900895DF92EF92FF9220
:1004A0000F931F93CF93DF93D82EAB0181E08D156F
:1004B00008F484C09B01ADECBCEC0E942B0EEC0157
:1004C000D695C795D695C795C031D10508F04EC0D1
:1004D0008E01CE01880F991F880F991F080F191FD1
:1004E000CA01801B910B8C01D0FAEE24E0F8F12CAC
:1004F0000024F694E7940794F694E7940794FE2C6E
:10050000E02C6894E7F8FF24FA946D2D6270660F72
:10051000660F660F6E2944E050E080E00E945800AC
:10052000209709F040C042C042E050E06FEF81E008
:100530000E945800F3942F2D332727FD3095C217C2
:10054000D30790F742E050E0602F81E00E9458000E
:10055000CF2DCF5FC13194F542E050E060E281E001
:100560000E945800CF5FC131BCF328C0ED2DE1706F
:10057000F0E00024F695E7950794F695E795079443
:10058000FE2FE02DE068FF6F6D2D6270660F660F25
:10059000660F6E2B44E050E080E00E94580000E0BF
:1005A00010E0CFE0D0E0FF24F394BECF42E050E073
:1005B000602F81E00E945800C2E0CECFDF91CF9142
:1005C0001F910F91FF90EF90DF9008951F93CF93AD
:1005D000DF93C82F883248F56830710518F4D62F9C
:1005E00010E209C06031710520F4162F1770DFEF9B
:1005F00002C0DFEF1FEF6C2F606844E050E080E046
:100600000E94580042E050E0612F81E00E945800B3
:100610006C2F606C44E050E080E00E94580042E0A3
:1006200050E06D2F81E00E945800DF91CF911F9123
:100630000895CF93DF93EA01683250F5982F9270B6
:10064000990F990F990F692B282F217030E0002402
:10065000369527950794369527950794322F202DA8
:1006600020683F6F622B44E050E080E00E94580019
:10067000C830D10538F442E050E06C2F81E00E9490
:10068000580006C042E050E06FEF81E00E94580041
:10069000DF91CF910895CF93DF93CDB7DEB7E49785
:1006A0000FB6F894DEBF0FBECDBF1C821B828B81BC
:1006B0009C8142977CF50B811C816B817C816F5FF3
:1006C0007F4F882777FD8095982F0E94160C2BED81
:1006D0003FE049EC50E40E94DB0C20E030E048E4CD
:1006E00053E40E947B0B0E94780B00521F4F20E0C6
:1006F00030E04EEF52E40E94DB0C0E94E30BD80185
:100700006C938B819C8101969C838B838B819C81D4
:1007100042978CF28FEF84BB81BB82BB88BB8CEF8E
:100720008BBB0E94AC000E94FA018DE78CBF8AE06F
:1007300083BF8BE687B986E086B980E680BF86B145
:10074000806E86B944E050E062E880E00E94580084
:100750008CE990E00E94990044E050E066EC80E073
:100760000E94580089EA90E00E94990086B38F3F6A
:10077000E9F386B38F3FE9F740E850E061E080E0BD
:100780000E9458001EA21FA218A619A61E8E1F8E18
:1007900018A219A21EA604E60DA711E018AB06E0E8
:1007A0000FA718E01DA307E00C8F11E01D8F412C4F
:1007B000512C320101E0088F1A82198289819A81B5
:1007C00001969A838983893C91050CF07BC14D8603
:1007D0005E866F86788A49865A866B867C86F42D7B
:1007E000E52D342C252C6D8A7E8A4D825E826F82A7
:1007F00078864B8A5C8A698A7A8A1F8AD62CC72CAB
:100800000CC0F82FE92FDA2ECB2E382C292CAD8AEC
:10081000BE8AEB8AFC8A098B1A8B349BFECFA98196
:10082000BA8184B195B1AA0FBB1FAE50BF4F8D9353
:100830009C93349A88B7826088BFA981BA81AA0F35
:10084000BB1FAE50BF4F8D919C918115904861F0B8
:10085000A981BA81AA0FBB1FAE50BF4F8D919C9149
:10086000803C9F4731F403C0E88CEF8A02C0F88CCB
:10087000FF8AA981BA81AA0FBB1FAE50BF4F8D91CD
:100880009C911197082E892F000C881F990B000C42
:10089000881F991F8D939C9389819A81819734F544
:1008A000A981BA8189819A8149815A81AA0FBB1F86
:1008B000BD016E507F4F880F991F8E509F4FDC01F6
:1008C0002D913C91429FC001439F900D529F900DEE
:1008D00011249595879595958795959587959595E7
:1008E000879595958795DB018D939C9389819A8156
:1008F000893A910554F1A981BA8189819A81298126
:100900003A81AA0FBB1FBD016E507F4F880F991F00
:100910008E509F4F49EC50E0421B530BDC012D9150
:100920003C91429FC001439F900D529F900D112416
:10093000959587959595879595958795959587959F
:1009400095958795DB018D939C93A9EEB0E08C91F2
:10095000A82FBB27A7FDB0952B893C8949895A89C7
:100960000E94370EDC01CB01689415F8B595A79568
:10097000979587951694D1F7AC01BD01ED80FE8067
:100980000F8118854E195F09600B710BA981BA811F
:10099000AA0FBB1FAE50BF4F8D919C91AA2797FD08
:1009A000A095BA2F7A018B01E80EF91E0A1F1B1FB2
:1009B000A8EEB0E08C91A82FBB27A7FDB095232D02
:1009C000322D4D895E890E94370E4B015C0168947F
:1009D00015F8B594A794979487941694D1F7298520
:1009E0003A854B855C85821A930AA40AB50AA981C7
:1009F000BA81AA0FBB1FAE50BF4F8D919C91AA2701
:100A000097FDA095BA2F880E991EAA1EBB1EAAEEAE
:100A1000B0E08C91A82FBB27A7FDB0952F2F3E2FBC
:100A20004D2D5C2D0E94370EAB01BC01689415F86A
:100A300075956795579547951694D1F78D859E8541
:100A4000AF85B889481B590B6A0B7B0BA981BA810A
:100A5000AA0FBB1FAE50BF4F8D919C91AA2797FD47
:100A6000A095BA2F840F951FA61FB71F29813A8121
:100A70002F5F3F4F3A8329834B894D835C895E8387
:100A800069896F834A89488739862A865D895B87A9
:100A90006E896C87FD87EE87DF86C88A293C310521
:100AA0000CF4AFCEED82FE820F8318871D2D0C2D26
:100AB0006C017D01E98F1A8F0B8FE52FF62F1B89B3
:100AC0000C8915C04D86598E6A8E7B8E342C252C50
:100AD000E62DF72D7301620153014201142D052DFE
:100AE000698A7A8A4D825E826F8278861F8AA50122
:100AF0009401C501B4010E943F0E69877A878B87F4
:100B00009C87232D322D4E2F5F2F632D722D8E2F1C
:100B10009F2F0E943F0E29853A854B855C85260FC5
:100B2000371F481F591F29873A874B875C87A501C4
:100B30009401632D722D8E2F9F2F0E943F0E9B01DB
:100B4000AC01E8EEF0E0A081BB27A7FDB0950E94C4
:100B5000370EDC01CB01689415F8B595A7959795EC
:100B600087951694D1F729853A854B855C85281B96
:100B7000390B4A0B5B0B29873A874B875C872D81A2
:100B80003E814F815885CA01B9010E943F0E4B0139
:100B90005C01212F302F49895A89612F702F842FB2
:100BA000952F0E943F0E860E971EA81EB91E2D81FE
:100BB0003E814F815885612F702F89899A890E94C3
:100BC0003F0E9B01AC01E9EEF0E0A081BB27A7FD41
:100BD000B0950E94370EDC01CB01689415F8B595ED
:100BE000A795979587951694D1F795018401081BD1
:100BF000190B2A0B3B0B0D831E832F833887A7010C
:100C00009601C701B6010E943F0E4B015C012D8584
:100C1000398D4A8D5B8D622F732F842F952F0E9403
:100C20003F0E860E971EA81EB91EA70196016D8560
:100C3000798D8A8D9B8D0E943F0E9B01AC01EAEE5F
:100C4000F0E0A081BB27A7FDB0950E94370EDC0124
:100C5000CB01689415F8B595A79597958795169447
:100C6000D1F785017401E81AF90A0A0B1B0BED860E
:100C7000FE860F87188BFF88F11002C0979A01C07B
:100C800097980D8D0111E3C18D819E81AF81B8854B
:100C9000EE8CFF8C08A119A120EEE21623E9F206E2
:100CA00024E002071105F0F130E2E31631EAF30621
:100CB00037E003071105C8F52EA13FA148A559A5A6
:100CC000E216F3060407150778F4E816F9060A0792
:100CD0001B0750F46C017D0182179307A407B50729
:100CE000B0F569017A0133C0EE8CFF8C08A119A11F
:100CF0002EA13FA148A559A52E153F054007510734
:100D0000E8F48E159F05A007B107E8F4CD80DE80DA
:100D1000EF80F884281739074A075B07C0F4690198
:100D20007A0115C07301620112C00F2EC12CF5E3C8
:100D3000DF2EFCE0EF2EF12CF02D09C0CE8CDF8CE5
:100D4000E8A0F9A004C0CE8CDF8CE8A0F9A08985CA
:100D50009A85AB85BC8581389A41A640B10510F0D3
:100D6000929801C0929A0D851E852F853889013889
:100D70001A412640310510F0909801C0909A51E830
:100D8000C5165AE1D50656E0E506F104A8F00BA118
:100D9000011101C091981BA11F5F1BA3CEA2DFA26E
:100DA000E8A6F9A6ED80FE800F811885EE8EFF8EF5
:100DB00008A319A31CA25EC30BA10230A0F41CA1BE
:100DC00011116FC0919ACEA2DFA2E8A6F9A6ED801C
:100DD000FE800F811885EE8EFF8E08A319A31CA636
:100DE0001AA21BA247C30CA101115BC01CA51F5F67
:100DF0001CA70AA1000F0AA31FA5112389F00BA1AC
:100E0000053608F044C01DA5011708F40DA70EA56E
:100E10001BA1011708F41EA70FA501500FA737C08B
:100E200018A91130A1F50DA5202F30E01EA5812FA6
:100E300090E0A901440F551F481759071CF5820F70
:100E4000931F959587958C8F803198F499279C01F5
:100E5000220F331F220F331F820F931F9595879503
:100E6000959587958DA31EA614E61DA706E00FA7EE
:100E70000EC01C8D1C5F1DA31EA604E60DA716E068
:100E80001FA705C01EA604E60DA716E01FA70BA10D
:100E90001C8D101718F40AA101600AA3919A1BA2D5
:100EA00003C01CA11F3F19F00CA10F5F0CA31CA1D4
:100EB000212F30E00DA1802F90E0019628173907EF
:100EC00021F542E050E06FEF81E00E9458006BA5F1
:100ED0006270660F660F660F1AA5612B0BA5017075
:100EE0000BAB1CAA8BA99CA9002496958795079407
:100EF000969587950794982F802D80689F6F682B13
:100F000044E050E080E00E9458001CA10DA11013A5
:100F100093C21CA5113029F40AA1011142C065E653
:100F200055C01CA5123039F40AA1E02FF0E0E856B4
:100F3000FF4F60814BC01CA5133039F40AA1E02F8C
:100F4000F0E0E057FF4F608141C01CA5143039F438
:100F50000AA1E02FF0E0E058FF4F608137C01CA5E8
:100F6000153039F40AA1E02FF0E0E05AFF4F60811C
:100F70002DC01CA51630B9F40AA10531B1F0033318
:100F8000B1F00833B1F00C30B1F00131B1F00631FD
:100F9000B1F00D32B1F00A30B1F00A31B1F460E4D1
:100FA00015C064E713C060E211C06EE20FC06CE2CE
:100FB0000DC06AE30BC06FE309C06DE207C068E2D1
:100FC00005C069E203C06FE201C060E242E050E0A8
:100FD00081E00E9458008AA58F5F1AA51F3008F48F
:100FE00038C20BA5802F90E00196817090788BA776
:100FF0009C01217033270024369527950794369558
:1010000027950794322F202D20683F6F82709927F3
:10101000880F991F880F991F880F991F622F682BBF
:1010200044E050E080E00E945800CEA2DFA2E8A693
:10103000F9A6ED80FE800F811885EE8EFF8E08A345
:1010400019A3FCA0FDA21AA61CA61AA213C282E034
:1010500090E09C838B838B819C8108970CF0C4C0AB
:1010600001E010E01A83098389819A81893C910506
:101070000CF055C073016201042D152DF62DE72DDE
:1010800004C0082D192DFA2DEB2DAB81BC81A05287
:10109000BF4FAC91AA0FBB0B202F312F4F2F5E2FCC
:1010A0000E94370E4B015C0199235CF40F2EFFE781
:1010B0008F2E912CA12CB12CF02D860E971EA81EE0
:1010C000B91E689416F8B594A794979487941694CB
:1010D000D1F78C189D08AE08BF08A981BA81AA0F64
:1010E000BB1FAE50BF4F8D919C91AA2797FDA09535
:1010F000BA2F880E991EAA1EBB1E89819A8101965D
:101100009A83898389819A81C02ED12EEF2EFE2E5B
:10111000893C91050CF4B5CF3F2E2E2E06C0042D30
:10112000152D362C272C53014201EB81FC81A501A2
:101130009401C501B4010E943F0E6B017C01202F78
:10114000312F432D522D602F712F832D922D0E9410
:101150003F0EC60ED71EE81EF91EA5019401602F92
:10116000712F832D922D0E943F0E9B01AC01E05206
:10117000FF4FA081BB27A7FDB0950E94370EDC0171
:10118000CB01689415F8B595A79597958795169412
:10119000D1F7A7019601281B390B4A0B5B0BCA013B
:1011A000B9010E94160C0E94420D0B811C8120E0A7
:1011B00030E040E250E40E94DB0C20E030E048E404
:1011C00053E40E947B0B0E94E80B7727802F82500C
:1011D0000E94E6028B819C8101969C838B838B818C
:1011E0009C8108970CF43CCF8BE090E09C838B8330
:1011F0008B819C8142970CF0C4C041E050E05A833F
:10120000498389819A81893C91050CF055C073010D
:101210006201042D152DF62DE72D04C0082D192D82
:10122000FA2DEB2DAB81BC81A052BF4FAC91AA0F20
:10123000BB0B202F312F4F2F5E2F0E94370E4B01FB
:101240005C0199235CF40F2EFFE78F2E912CA12CCB
:10125000B12CF02D860E971EA81EB91E689416F8A4
:10126000B594A794979487941694D1F78C189D08F9
:10127000AE08BF08A981BA81AA0FBB1FAE50BF4FED
:101280008D919C91AA2797FDA095BA2F880E991E43
:10129000AA1EBB1E89819A8101969A8389838981BE
:1012A0009A81C02ED12EEF2EFE2E893C91050CF492
:1012B000B5CF3F2E2E2E06C0042D152D362C272CF3
:1012C00053014201EB81FC81A5019401C501B401E8
:1012D0000E943F0E6B017C01202F312F432D522D98
:1012E000602F712F832D922D0E943F0EC60ED71EA8
:1012F000E81EF91EA5019401602F712F832D922DF8
:101300000E943F0E9B01AC01E052FF4FA081BB2722
:10131000A7FDB0950E94370EDC01CB01689415F84B
:10132000B595A795979587951694D1F7970186015E
:10133000081B190B2A0B3B0BC901B8010E94160CA4
:101340000E94420D0B811C8120E030E040E250E41D
:101350000E94DB0C20E030E048E453E40E947B0B69
:101360000E94E80B7727802F82500E94E6028B8133
:101370009C8101969C838B838B819C8142970CF48A
:101380003CCF69857A858B859C850E94160C0E94CE
:10139000420D20E030E040E250E40E94DB0C20E00F
:1013A00030E048E453E40E947B0B0E94E80B77276F
:1013B00086E00E94E6026D817E818F8198850E9481
:1013C000160C0E94420D20E030E040E250E40E9402
:1013D000DB0C20E030E048E453E40E947B0B0E94E9
:1013E000E80B772787E00E94E6026D857E858F8572
:1013F00098890E94160C0E94420D20E030E040E2E5
:1014000050E40E94DB0C20E030E048E453E40E940A
:101410007B0B0E94E80B772788E00E94E60244E0FD
:1014200050E067EC80E00E94580042E050E06EE53A
:1014300081E00E9458001EC0CEA2DFA2E8A6F9A655
:10144000ED80FE800F811885EE8EFF8E08A319A314
:1014500011C0CEA2DFA2E8A6F9A6ED80FE800F8122
:101460001885EE8EFF8E08A319A38AA7FCA0FDA203
:101470001CA61AA286B38F3F09F49EC916B3112386
:101480000CF447C00D8D013079F440E850E061E084
:1014900080E00E94580044E050E060E880E00E9454
:1014A00058001BA61AA620C18AE29CE2AAE0B0E07E
:1014B000B79905C00197A109B109D1F704C0892BDB
:1014C0008A2B8B2B59F440E850E061E080E00E94C9
:1014D000580016FF23C001E00D8FBAC00C8D0230FA
:1014E00010F001500C8F0C8D003178F4802F90E0BB
:1014F0009C01220F331F220F331F820F931F9595DC
:101500008795959587958DA3EFC00C8D0C5F0DA3E6
:10151000EBC016FD9DC01D8D113081F440E850E0F8
:1015200061E080E00E94580044E050E060E880E024
:101530000E9458001BA61AA61D8ED2C08AE29CE209
:10154000AAE0B0E0B69905C00197A109B109D1F7A9
:1015500005C0892B8A2B8B2B09F05DC0E8A8E11010
:1015600027C00C8D003178F4802F90E09C01220F71
:10157000331F220F331F820F931F959587959595E3
:1015800087958DA303C01C8D1C5F1DA344E050E014
:1015900067EC80E00E9458008FEA90E00E9499007A
:1015A0001EA604E60DA711E018AB06E00FA70BC0BE
:1015B00044E050E067EC80E00E94580089EB90E046
:1015C0000E94990018AA1AA5173028F00BA501301F
:1015D00011F41BA61AA66BA56270660F660F660F44
:1015E0001AA5612B0BA5017009AB1AAA89A99AA9A2
:1015F0000024969587950794969587950794982F3C
:10160000802D80689F6F682B44E050E080E00E944E
:1016100058001D8E65C01C8D143610F41F5F1C8F82
:101620000C8D003180F4802F90E09C01220F331F3D
:10163000220F331F820F931F959587959595879558
:101640008DA31D8E4DC01C8D1C5F1DA31D8E48C01B
:1016500010FD46C040E850E061E080E00E94580084
:1016600044E050E060E880E00E94580083EC90E0A5
:101670000E94990088EE93E00E94310186EC90E090
:101680000E9499008C8D0E94FF0044E050E060ECC5
:1016900080E00E9458008CEC90E00E9499008DA59B
:1016A0000E94FF008FEC90E00E9499008EA50E949E
:1016B000FF0008A9013029F483ED90E00E94990011
:1016C00004C089ED90E00E94990086B38F3FE9F74E
:1016D00040E850E061E080E00E9458001BA61AA696
:1016E00086B38F3FE9F768C816FF28CF1D8EB0CFAD
:1016F000F0D0E39526C10CD013C1E3D040F0DAD08E
:1017000030F021F45F3F19F0CCC051114EC1CFC071
:1017100029D198F39923C9F35523B1F3951B550BA0
:10172000BB27AA2762177307840738F09F5F5F4FB4
:10173000220F331F441FAA1FA9F333D00E2E3AF0F5
:10174000E0E830D091505040E695001CCAF729D00F
:10175000FE2F27D0660F771F881FBB1F261737075E
:101760004807AB07B0E809F0BB0B802DBF01FF278E
:1017700093585F4F2AF09E3F510568F092C015C103
:101780005F3FECF3983EDCF3869577956795B795C8
:10179000F7959F5FC9F7880F911D9695879597F9E3
:1017A0000895E1E0660F771F881FBB1F621773075C
:1017B0008407BA0720F0621B730B840BBA0BEE1F71
:1017C00088F7E095089504D06894B111EEC00895AB
:1017D000D1D088F09F5790F0B92F9927B751A0F03A
:1017E000D1F0660F771F881F991F1AF0BA95C9F7B5
:1017F00012C0B13081F0D8D0B1E00895D5C0672FC4
:10180000782F8827B85F39F0B93FCCF38695779564
:101810006795B395D9F73EF490958095709561954D
:101820007F4F8F4F9F4F0895E89409C097FB3EF478
:1018300090958095709561957F4F8F4F9F4F99231D
:10184000A9F0F92F96E9BB279395F695879577959B
:101850006795B795F111F8CFFAF4BB0F11F460FF5B
:101860001BC06F5F7F4F8F4F9F4F16C0882311F0B3
:1018700096E911C0772321F09EE8872F762F05C0C7
:10188000662371F096E8862F70E060E02AF09A9562
:10189000660F771F881FDAF7880F9695879597F957
:1018A000089597F99F6780E870E060E008959FEFE2
:1018B00080EC089500240A941616170618060906E7
:1018C000089500240A9412161306140605060895B6
:1018D000EECF50D0E8F3E894E0E0BB279F57F0F05C
:1018E0002AED3FE049EC06C0EE0FBB0F661F771FE5
:1018F000881F28F0B23A62077307840728F0B25AAB
:10190000620B730B840BE3959A9572F7803830F471
:101910009A95BB0F661F771F881FD2F7904852C158
:10192000092E0394000C11F4882352F0BB0F40F4ED
:10193000BF2B11F460FF04C06F5F7F4F8F4F9F4F2D
:101940000895EF93E0FF06C0A2EA2AED3FE049ECDC
:101950005FEBE3D0E5DF0F90039401FC9058E4E5E2
:10196000F0E043C157FD9058440F551F59F05F3FB9
:1019700071F04795880F97FB991F61F09F3F79F0B1
:1019800087950895121613061406551FF2CF469533
:10199000F1DF08C0161617061806991FF1CF8695B5
:1019A0007105610508940895E894BB276627772799
:1019B000CB0197F908950BD0B3CF7CDF28F081DFFE
:1019C00018F0952309F06DCF72CF1124EECFCADF46
:1019D000A0F3959FD1F3950F50E0551F629FF00142
:1019E000729FBB27F00DB11D639FAA27F00DB11D9B
:1019F000AA1F649F6627B00DA11D661F829F222724
:101A0000B00DA11D621F739FB00DA11D621F839FAA
:101A1000A00D611D221F749F3327A00D611D231F80
:101A2000849F600D211D822F762F6A2F11249F57CE
:101A300050408AF0E1F088234AF0EE0FFF1FBB1FF1
:101A4000661F771F881F91505040A9F79E3F510590
:101A500070F027CFAACF5F3FECF3983EDCF386957A
:101A600077956795B795F795E7959F5FC1F7FE2B3B
:101A7000880F911D9695879597F9089511F40EF4A6
:101A800016CF9EC077DFD0F39923D9F3CEF39F57BB
:101A9000550B87FFA3D00024A0E640EA90018058B0
:101AA0005695979528F4805C660F771F881F20F065
:101AB00026173707480730F4621B730B840B202965
:101AC00031294A2BA69517940794202531254A27BA
:101AD00058F7660F771F881F20F02617370748072B
:101AE00030F4620B730B840B200D311D411DA0954A
:101AF00081F7B901842F9158880F9695879508959D
:101B0000D9DE30F0DEDE20F031F49F3F11F41EF418
:101B1000CECE0EF4E095E7FBC4CEE92F23DF80F3B1
:101B2000BA17620773078407950718F071F49EF5DA
:101B30003BCF0EF4E0950B2EBA2FA02D0B01B9016F
:101B400090010C01CA01A0011124FF27591B99F033
:101B5000593F50F4503E68F11A16F040A22F232F3F
:101B6000342F4427585FF3CF469537952795A7958F
:101B7000F0405395C9F77EF41F16BA0B620B730B36
:101B8000840BBAF09150A1F0FF0FBB1F661F771FA7
:101B9000881FC2F70EC0BA0F621F731F841F48F45C
:101BA000879577956795B795F7959E3F08F0B3CFE2
:101BB0009395880F08F09927EE0F979587950895CC
:101BC0009F3F31F0915020F4879577956795B795B1
:101BD000880F911D9695879597F9089591505040DB
:101BE000660F771F881FD2F708959F938F937F9377
:101BF0006F93FF93EF939B01AC01DDDEEF91FF91BB
:101C000005D02F913F914F915F91D5CEDF93CF9328
:101C10001F930F93FF92EF92DF927B018C016894E8
:101C200005C0DA2EEF01D3DEFE01E894A5912591DF
:101C3000359145915591AEF3EF016FDFFE019701AC
:101C4000A801DA9479F7DF90EF90FF900F911F9140
:101C5000CF91DF910895A29FB001B39FC001A39FD0
:101C600001D0B29F700D811D1124911D0895B7FF01
:101C70000C944F0E0E944F0E821B930B0895DB01B4
:101C80008F939F930E944F0EBF91AF91A29F800DA3
:101C9000911DA39F900DB29F900D112408950E9455
:101CA0002B0EA59F900DB49F900DA49F800D911DAC
:081CB00011240895F894FFCF00
:101CB80035345F335F5F5F325F5F2A5F5F5F5F313D
:101CC800362D2F5F5F5F5F5F375F5F5F385F39304B
:101CD800687666756C61706A627863797A716F6824
:101CE80073757277646B676F69616E6D4D6F727330
:101CF800654465636F64657200444B33504B007CE8
:101D080053796E63206F6E20007C53796E63206F69
:101D1800666600663D00206469743D006D3D0020E4
:101D28004D3D002053594F4E002053594F46000057
:00000001FF
